:020000009C283A
:08000800FF00030E8301A000BC
:100010000A08A1008A010408A2000E280313831213
:10002000861B1828FA0A04307A0603192128192891
:10003000FA01061A3428FB0A04307B0603192B2820
:1000400035283030F400F201F501F60A3C3076062E
:10005000031D3528F6013030F400F201F70A0C30A8
:1000600077060319F7013528FB010B1D92280B11A8
:10007000FF308100F40A3C307406031D572801301C
:10008000F202031845280230F200F401F50A3C3070
:100090007506031D5728F501F60A3C307606031D48
:1000A0005728F601F70A0C3077060319F701F20812
:1000B000031D61280F3085007708F9007608F800E5
:1000C000922879087218780883169B001C147218FD
:1000D0007528F908031D6F2812309A0075280A3018
:1000E0001A0203187528F0309A048030F0000030AE
:1000F000F1001E307402031882289A0E0030F000BE
:100100004030F1000F309A057008721871081A0417
:10011000831285004030740783169B001C141A0854
:10012000831295008B162208840021088A00200E75
:100130008300FF0E7F0E09008030F0004030F10098
:100140000230F200F401F501F601F701F801F901BE
:10015000FA01FB01FF30A400FF30A5003030D720AA
:100160009730D5208312031307309F00640081016C
:1001700083166F3081006400683081008312FF3085
:10018000810083168E15FF3092008312950197121D
:100190001712043092000F3097000B118B168B173B
:1001A000CF3085000000D228D428A500D928A4008B
:0E01B000DC2825086600080024086500080009
:02400E00703F01
:024200000000bc
:024202000100b9
:024204000200b6
:024206000300b3
:024208000400b0
:02420a000500ad
:02420c000600aa
:02420e000700a7
:024210000800a4
:024212000900a1
:02421400100098
:02421600110095
:02421800120092
:02421a0013008f
:02421c0014008c
:02421e00150089
:02422000160086
:02422200170083
:02422400180080
:0242260019007d
:02422800200074
:02422a00210071
:02422c0022006e
:02422e0023006b
:02423000240068
:02423200250065
:02423400260062
:0242360027005f
:0242380028005c
:02423a00290059
:02423c00300050
:02423e0031004d
:0242400032004a
:02424200330047
:02424400340044
:02424600350041
:0242480036003e
:02424a0037003b
:02424c00380038
:02424e00390035
:0242500040002c
:02425200410029
:02425400420026
:02425600430023
:02425800440020
:02425a0045001d
:02425c0046001a
:02425e00470017
:02426000480014
:02426200490011
:02426400500008
:02426600510005
:02426800520002
:02426a005300ff
:02426c005400fc
:02426e005500f9
:024270005600f6
:024272005700f3
:024274005800f0
:024276005900ed
:02428000f0004c
:02428200ed004d
:02428400e50053
:02428600d9005d
:02428800c8006c
:02428a00b3007f
:02428c009d0093
:02428e008400aa
:024290006b00c1
:024292005200d8
:024294003b00ed
:024296002700ff
:0242980016000e
:02429a000a0018
:02429c00000020
:02429e0000001e
:0242a0000a0012
:0242a200160004
:0242a4002700f1
:0242a6003b00db
:0242a8005200c2
:0242aa006b00a7
:0242ac0084008c
:0242ae009d0071
:0242b000b30059
:0242b200c80042
:0242b400d9002f
:0242b600e50021
:0242b800ed0017
:0242ba00f00012
:0242bc00f00010
:0242be00ed0011
:0242c000e50017
:0242c200d90021
:0242c400c80030
:0242c600b30043
:0242c8009d0057
:0242ca0084006e
:0242cc006b0085
:0242ce0052009c
:0242d0003b00b1
:0242d2002700c3
:0242d4001600d2
:0242d6000a00dc
:0242d8000000e4
:0242da000000e2
:0242dc000a00d6
:0242de001600c8
:0242e0002700b5
:0242e2003b009f
:0242e400520086
:0242e6006b006b
:0242e800840050
:0242ea009d0035
:0242ec00b3001d
:0242ee00c80006
:0242f000d900f3
:0242f200e500e5
:0242f400ed00db
:0242f600f000d6
:00000001FF
